:10000300E4F512F5130513E51370020512E4B513B5
:10001300F4E512B420EF7FA41202447FBF1202441E
:10002300E4F5147F641202750514E514C3940340C8
:10003300F27FA4120244751000750F00750E00754F
:100043000D007511FF7F887DFC1202ED7F907D0806
:100053001202ED7F917D081202ED20932B7F151282
:1000630002F88F117FC9E511C4540FFD1202ED7F11
:10007300C8E511540FFD1202ED3093FD75100075A4
:100083000F00750E00750D007A0079007800E510F9
:100093002401F510EA350FF50FE9350EF50EE835B5
:1000A3000DF50DE51160167F007E007D037C00AB2E
:1000B30010AA0FA90EA80DC31202D0409D7F887D00
:1000C300FF1202EDE4F51474082514F8E4F6E514C0
:1000D3002480FF74082514F8E6FD1202ED0514E5EB
:1000E30014C3940540E1E50CC3940250710508E57F
:1000F30008D394094033E4F5080509E509D39409C5
:100103004027E4F509050AE50AD39409401BE4F501
:100113000A050BE50BD39409400FE4F50B050CE539
:100123000CD394094003E4F50C7F80AD081202ED73
:10013300E50870B27F81AD091202EDE50970A77F72
:1001430082AD0A1202EDE50A709C7F83AD0B1202A9
:10015300EDE50B70917F84AD0C1202ED80887F96E4
:100163001202757FA41202447F977D491202ED7F2C
:1001730050120275E4F5147FA21202447F0C12029E
:10018300750514E514C3941740EDE4F5147FA31229
:1001930002447F0C1202750514E514C3941740ED55
:1001A300E4F5147FA11202447F80AD141202ED7FA7
:1001B300321202750514E514C3941040E67F9612BB
:1001C30002757FA4120244E4F5147FA01202447F57
:1001D300CFAD141202ED7F321202750514E514C37C
:1001E300941040E67F961202757515FFE4F514E549
:1001F30015C313F5157F98FD1202ED7F6412027586
:100203000514E514C3940640E67F987DFF1202EDC2
:100213007F641202757FA4120244E4F514E514C34B
:10022300944040030200037FE0AD141202ED7FC04F
:10023300E51414FD1202ED7F14120275051480DD1E
:010243002298
:0B02ED008D16120244AF1612024422CC
:0702F8001202441202A422CD
:100244008F17C2941202FFE4F518E51730E704D2C1
:10025400928002C292D295120306C295120306E559
:100264001725E0F5170518E518C3940840DCC29279
:010274002267
:1002A400D2921202FFE4F516D295120306E5172541
:1002B400E0F517309203431701C2951203060516A1
:0C02C400E516C3940840E1C292AF172277
:0702FF00E4FF0FBF30FC22F9
:07030600E4FF0FBF08FC2219
:100275008F16E4F517E517C395165022E4F518F522
:10028500192093031200000519E51970020518C31A
:0F029500E5199490E518940340E7051780D722E8
:030000000202E118
:0C02E100787FE4F6D8FD75811902000357
:1002D000EB9FF5F0EA9E42F0E99D42F0E89C45F084
:0102E00022FB
:00000001FF
